:100000001BC033C0C8C231C030C02FC0D7C12DC043
:100010002CC02BC02AC044544D46204465636F64F5
:100020006572206279207777772E696E66696469D8
:10003000676D2E6E6574000011241FBECFEDCDBF1D
:1000400010E0A0E6B0E0E2E0F6E003C0C89531962B
:100050000D92A036B107D1F710E0A0E6B0E001C0E4
:100060001D92AA37B107E1F79DC0CACF982F869598
:100070008EBBE09A90FF05C08DB399278F7090706A
:1000800008958DB382958F70992708950895CF9321
:10009000DF93CDB7DEB722970FB6F894DEBF0FBE61
:1000A000CDBF9FEF97BB813011F4959A01C0959811
:1000B00068BB19821A8289819A81C29730F489813A
:1000C0009A81019689839A83F6CF969A19821A8229
:1000D00089819A81C29730F489819A8101968983B6
:1000E0009A83F6CF969819821A8289819A81883CE0
:1000F000910530F489819A81019689839A83F5CF9D
:1001000017BA22960FB6F894DEBF0FBECDBFDF91AF
:10011000CF9108955D9BFECF8CB908950F931F93E7
:10012000CF93DF93D92FC82F00E060E8802FAFDF97
:10013000FD2FEC2FC895802D8823B9F0FD2FEC2FD3
:10014000C895102D1CB9003119F460EC80E09FDFD8
:10015000612F81E09CDF21960F5F5D9BFECFFD2F1D
:10016000EC2FC895802D882349F7DF91CF911F91FF
:100170000F9108958F3019F480E290E008958A304D
:1001800019F480E390E008958B3019F48AE290E04E
:1001900008958C3019F483E290E0089580639927E4
:1001A00008950895CFEDD0E0DEBFCDBFF89417BA23
:1001B00080E781BBC49886E189B988E08AB983E089
:1001C00083BF82E089BF80E88BBF8CE285BF80EC73
:1001D0008ABF109264008091640048DF8F3039F04C
:1001E000809164008F5F809364008F3FA1F78091BE
:1001F00064008093780083E18093620081E08093C3
:100200007300682F80E043DF62E080E040DF68E356
:1002100080E03DDF6CE080E03ADF66E080E037DFE1
:100220008DE078DF8AE076DF86E190E077DF8DE0B1
:1002300071DF8AE06FDF10927900809179009091F0
:100240006400890F8F5F12DF95DF64DF8091790092
:100250008F5F809379008F3F81F78DE05BDF8AE0CD
:1002600059DF78948895FECF1F93CF93C82F162F10
:100270008A3020F460E281E00ADF04C061E381E0BB
:1002800006DFCA50C0636C2F81E001DF6DE281E0C0
:10029000FEDEC1E0809178008C0F811B8E50E6DE7F
:1002A00069DF682F81E0F3DECF5FCE3098F3CF9126
:1002B0001F91089561E381E0EADE69E381E0E7DE12
:1002C0006DE281E0E4DE1092790080917200882373
:1002D00091F080917900E82FFF27EB59FF4F608163
:1002E00081E0D5DE809179008F5F809379009091D5
:1002F0007200891770F30895CF93C82F609173002F
:100300006130A1F4809172008D3080F410927300FE
:100310001092600083E18093620080E0B8DE60E0CC
:1003200082E1A2DF60EC80E0B2DEC4DF8091720087
:100330008D30A8F161E080E0AADE61E381E0A7DE14
:1003400068E381E0A4DE6DE281E0A1DE109272003C
:1003500080917200E82FFF27EB59FF4F608181E009
:1003600096DE809172008F5F809372008E3080F3F2
:1003700060EC80E08CDE61E381E089DE69E381E0AE
:1003800086DE6DE281E083DE10927200809164006F
:10039000809378001092600083E1809362006C2F5C
:1003A00081E075DE80917200E82FFF27EB59FF4F47
:1003B000C0838F5F80937200CF9108951F920F9238
:1003C0000FB60F9211241F932F933F934F935F9378
:1003D0006F937F938F939F93AF93BF93CF93EF933D
:1003E000FF93809B0EC086E180937400809176001D
:1003F000863120F48F5F8093760042C010926100B6
:100400003FC01092760080917400882321F08150C3
:100410008093740035C0C0916100CC2389F5809130
:100420006200833168F511E010937300810F8093AF
:100430006200612F8C2F2BDE809160008D50909197
:100440006200682F892F81500FDF60EC8C2F1FDE38
:1004500090916200933131F0809160008A51682F51
:10046000892F02DF809160008D5080936000809121
:100470006200833119F41EDFC09373001093610092
:1004800080B38695869580FF0EC086E180937500C7
:1004900080917700863120F48F5F8093770036C09B
:1004A0001092630033C0109277008091750088230A
:1004B00021F081508093750029C0C0916300CC2346
:1004C00029F580916200833008F111E010937300E8
:1004D000815080936200612F8C2FD9DD8091600064
:1004E000835F90916200682F892F8150BDDE60ECA0
:1004F0008C2FCDDD6091600080916200B5DE80912F
:100500006000835F8093600010936300FF91EF9120
:10051000CF91BF91AF919F918F917F916F915F919B
:100520004F913F912F911F910F900FBE0F901F90F1
:100530001895F894E199FECF86958EBB6DBBE29A33
:10054000E19A78940895CF93C82F8091640080FF3A
:1005500016C081508BDD682F6295607F6C2B809177
:100560006400E7DF809164008F5F809364008F5F99
:100570007DDD682F606F80916400DBDF0AC0C2956B
:10058000C07FCF606C2FD5DF809164008F5F809338
:100590006400CF9108951F920F920FB60F9211240D
:1005A0000F931F932F933F934F935F936F937F937B
:1005B0008F939F93AF93BF93EF93FF93F89417BAE2
:1005C000949A000016B394981F70812FD3DD082FE2
:1005D00093DE812FB8DF802F9DDD7894FF91EF911E
:1005E000BF91AF919F918F917F916F915F914F914B
:1005F0003F912F911F910F910F900FBE0F901F9061
:0206000018954B
:00000001FF
